:020000040000FA
:0400000080314E28D5
:100008007E1480310B1D4C280130F0007008200050
:10001800AA070130F0007008A9070130F000700845
:10002800A7070130F0007008A60725082702031C5F
:1000380032282C0012082000240203182728013037
:100048002C009202302824082C00120203183028B1
:100058000130F000700892072000A7012508260249
:10006800031C4B282C0015082000230203184028E5
:1000780001302C009502492823082C00150203188A
:1000880049280130F000700895072000A6010B11DF
:100098007E10090080315028F901FA012000A001E2
:1000A800A101A201A301A401A501A601A701A8011C
:1000B800A901AA017E1020008031622821001915AB
:1000C8009911191699168C1624008C16210095136F
:1000D800951295158B168B171E129E121E139E17BE
:1000E8000C160E148E140E1523000C160E148E14F6
:1000F8000E1521001D148E128E11FF3020009B005A
:1001080004309C002C00931713179617161720001D
:100118008C1A9028A2019228A201A20A2208031D83
:100128009D28C830AB002B08F900A801A80AA50132
:10013800AC282203031DAC28FA30AB002B08F900C9
:100148001030AB002B08A8000430AB002B08A5002A
:1001580079082A02031CDA28A001A101FA0128085B
:100168007A020318C6288131092180312000AB00AA
:10017800AC012B08A0072C08A13D0130AB002B08CF
:10018800FA07B3287A08AB00AC012B08F1002C0859
:10019800F2002108F4002008F30081314E2180315B
:1001A80071082000AD002D08A400AA0179082902D1
:1001B800031C8B28A001A101FA0128087A02031860
:1001C800F4288131092180312000AB00AC012B08D3
:1001D800A0072C08A13D0130AB002B08FA07E12845
:1001E8007A08AB00AC012B08F1002C08F2002108BA
:1001F800F4002008F30081314E218031710820007D
:10020800AD002D08A300A9018B2821001D159D15FF
:100218001D129D149D180E291B080139F100710843
:10022800F3001D119D111D169D149D1819291B08F9
:1002380001390907F1007108F3071D159D111D16F5
:100248009D149D1825291B080139F1000130F1354D
:10025800FF3E031D2B297135F2007208F3071D11AB
:100268009D151D169D149D1837291B080139F1008D
:100278000230F135FF3E031D3D297135F200720849
:10028800F3077308F1000330F135FF3E031D4829D9
:1002980071350800F601F7017108720403197D2908
:1002A800F801F80AF21B62290130F135F20D890BC9
:1002B80059290130F5007508F80756290130F63537
:1002C800F70D890B632972087402031D6D297108E3
:1002D8007302031C74297108F3027208F43B761444
:1002E8000130F236F10C890B75290130F802031D33
:0C02F80062297708F2007608F100080087
:020000040001F9
:04000E00A4C9CFFFB3
:00000001FF
